:100000005828A40014200C080D04031953284D206F
:1000100084132408800664000D280E288C0A031916
:100020008D0F0B2880065328FF3A8417800553282C
:100030008F018E00FF308E07031C8F07031C53288F
:1000400003308D00DF3026201A288D01E83E8C0019
:100050008D09FC30031C2F288C0703182C288C07D3
:1000600064008D0F2C280C1835288C1C39280000B2
:10007000392808008E0001303D2894000F080D0239
:10008000031D44280E080C02043003180130031924
:1000900002301405031DFF3053288C098D098C0A8A
:1000A00003198D0A080083130313831264000800E8
:1000B00083168501113086008312850186017C2814
:1000C0007830AC000F308500000000000000000018
:1000D000000000000000000000000030850000006B
:1000E0000000000000000000000000000000000010
:1000F0000000AC0B62280800BE308C008D01063079
:100100008400083001200330AD000130A800A901AF
:1001100028088C0029088D008F0105303A20031D26
:10012000A528861683168612831201308F00F430BC
:100130001920861283168612831201308F00F43044
:100140001920A80A0319A90F88280130A800A901BD
:1001500028088C0029088D0013308F0088303A2041
:10016000031DBB286400061CEB2801301820A80AD8
:100170000319A90FA82886168316861283126020F9
:100180006020602060206020053018206020602002
:1001900060206020602005301820602060206020F2
:1001A00060206020053018206020602060206020E2
:1001B00008301820602003301820602060200830AC
:1001C00018206020033018206020602086128316DB
:1001D00086128312A5280330182064000618A5286B
:1001E0000330182064000618A528AD036400013010
:1001F0002D02031C6C29061783160613831286171B
:1002000083168613831296308C008D01063084008D
:1002100008300120193018208C308C008D010630F8
:100220008400083001201930182096308C008D0190
:100230000630840008300120193018208C308C00E2
:100240008D0106308400083001201930182001305B
:10025000A800A90128088C0029088D008F011930F9
:100260003A20031D6B29061783160613831286177F
:10027000831686138312B4308C008D0106308400FF
:100280000830012032301820BE308C008D0106303D
:10029000840008300120323018200613831606131C
:1002A00083128613831686138312B4308C008D015B
:1002B000063084000830012032301820BE308C0017
:1002C0008D01063084000830012032301820A80A41
:1002D0000319A90F2A29BB280130A800A901280861
:1002E0008C0029088D008F0164303A20031DD42929
:1002F000061783160613831286138316861383123A
:1003000078308C008D0106308400083001201930CF
:10031000182082308C008D010630840008300120C6
:100320001930182078308C008D0106308400083098
:1003300001201930182082308C008D010630840095
:100340000830012019301820061383160613831273
:100350008617831686138312B4308C008D01063005
:1003600084000830012019301820BE308C008D0127
:10037000063084000830012019301820B4308C0079
:100380008D01063084000830012019301820BE305D
:100390008C008D01063084000830012019301820AF
:0E03A000A80A0319A90F6F297C286300D5292C
:02400E00FE3F73
:00000001FF
